:1000000012C02CC02BC02AC029C028C027C026C0BF
:1000100025C024C023C022C021C020C01FC01EC0D4
:100020001DC01CC01BC011241FBECFE5D4E0DEBF25
:10003000CDBF10E0A0E6B0E0E2EFF1E002C0059035
:100040000D92A237B107D9F710E0A2E7B0E001C0E6
:100050001D92A237B107E1F73ED0C9C0D1CF2AEF38
:1000600030E004C0F9013197F1F701970097D1F71B
:100070000895BB9ABD9A8A98BA9AA19AA39A0895AC
:10008000C29AC39AC59880B3A99A0895C598C29890
:1000900020E0C598C59897FF02C0C39A01C0C398D5
:1000A000C59AC59A2F5F203119F0880F991FF1CF9B
:1000B000C598C29A089590E08299FECF829BFECFA8
:1000C00087FF02C0A99A01C0A9989F5F983011F0DC
:1000D000880FF2CF0895EF92FF920F931F93CF9363
:1000E000DF93BB9ABD9A8A98BA9AA19AA39AC29AA8
:1000F000C39AC59880B3A99AAB9A24E630E04AEF38
:1001000050E003C0CA010197F1F7215030408FEF52
:100110002F3F3807B9F780E09CECB8DF82E790E921
:10012000B5DF80E496EAB2DF80E490EDAFDF87E4EC
:1001300098ECACDF80E292ECA9DF81E090ECA6DFE6
:1001400080E090EBA3DF00E04AEFE42EF12CAB9AC5
:1001500089E390EC9BDF8AEAAEDF8AEAACDF8AEAC9
:10016000AADF8DE2A8DF84EDA6DFC0E6D0E010E0D4
:100170008881A1DF8991180F20E0C037D207C1F72D
:10018000812F99DF8AEA97DF8AEA95DF81E090EC98
:100190007DDFAB9884EF91E003C0F7013197F1F771
:1001A00001972FEF8F3F9207C1F70F5F802F64E613
:1001B00012D0805D80936D00802F0DD0292F892F64
:1001C0006AE009D0805D80936E00822F04D0905D3C
:1001D00090936F00BCCF991B79E004C0991F9617CC
:1001E00008F0961B881F7A95C9F780950895F894B2
:0201F000FFCF3F
:1001F2000A0D41546D65676131360A0D202D2D2D92
:020202000000FA
:00000001FF
